:020000040000FA
:020000000428D2
:08000800FF30A2000730A40044
:100010000830A4000830A5000130A6000530A70074
:100020000530A70080201F20221585200230A8005F
:10003000A010201545201E08242016281E28A314D1
:1000400023088500A2108628A8008B1B28282A28B0
:100050008B1325282808A9000B30AA003828013066
:10006000AB002408AC00AC0B3328AB0B31280800E4
:1000700003100318A314031CA310230885002F20CA
:100080000314A90CAA0B39280800A808031D4B2843
:100090000130A9005F282808013C031D52280230C6
:1000A000A9005F282808023C031D59280430A90034
:1000B0005F282808033C031D5F280830A900831629
:1000C0002908103E9F0083122808AB000230AC00C4
:1000D0009320AA002A08A80028089F00A01C7228C4
:1000E0001F1773281F13201D77289F1378289F1729
:1000F0001F1401308A209F149F1C7F287C28080031
:100100008316FF239000831208008728872822087F
:1001100065000800AB000F30AC00AC0B8D28000070
:10012000AB0B8B280800AC002C08003C031C992862
:100130009F280310AB0D01302C02AC0094282B0833
:020140000800B5
:02400E00C211DD
:00000001FF
